:100000008A110A120528000009000730990083169A
:100010000510851005118312BC30A0000230A1002C
:1000200052212F20AC012C080A3C031C2B28AD01C7
:100030002D083B3C031C2528E830A0000330A1001C
:1000400052210130AD07031C18281F3083050130F1
:10005000AC07031C13281F3083050C282E28051419
:100060002030A0000330A10052215D20FA20592049
:10007000FA20CA20FA20AE20FA204C20FA2096203E
:100080009030A0000130A100522105102C30A000BA
:100090000130A100522108001E212F2108002F212C
:1000A0001E211E211E2108002F211E212F211E216D
:1000B00008002F211E211E2108001E2108001E21DC
:1000C0001E212F211E2108002F212F211E21080073
:1000D0001E211E211E211E2108001E211E21080096
:1000E0001E212F212F212F2108002F211E212F21FA
:1000F00008001E212F211E211E2108002F212F2143
:1001000008002F211E2108002F212F212F21080058
:100110001E212F212F211E2108002F212F211E21DA
:100120002F2108001E212F211E2108001E211E2123
:100130001E2108002F2108001E211E212F2108004A
:100140001E211E211E212F2108001E212F212F21BB
:1001500008002F211E211E212F2108002F211E21E2
:100160002F212F2108002F212F211E211E210800C1
:100170002F212F212F212F212F2108001E212F2158
:100180002F212F212F2108001E211E212F212F2159
:100190002F2108001E211E211E212F212F210800A2
:1001A0001E211E211E211E212F2108001E211E217D
:1001B0001E211E211E2108002F211E211E211E216D
:1001C0001E2108002F212F211E211E211E21080083
:1001D0002F212F212F211E211E2108002F212F2109
:1001E0002F212F211E21080005114630A000A1015A
:1001F0005221080005114630A000A10152214630CD
:10020000A000A10152214630A000A1015221080006
:1002100005114630A000A10152214630A000A101E5
:1002200052214630A000A10152214630A000A10178
:1002300052214630A000A1015221080005150530C9
:1002400084000230AA009930A0000230A1003530AD
:10025000A2000030A3008D210511F420080005152F
:10026000053084000230AA009930A0000230A100BD
:10027000D230A2000030A3008D210511F420080027
:100280000515053084000230AA009930A000023024
:10029000A100EE30A2000230A3008D210511F42050
:1002A00008005129A00803195D296421A00300005A
:1002B00000000000000000005229A10803190800F6
:1002C0006421A103A00352290C30A500A50B6629C7
:1002D000000000001230A200A20B732975217521C5
:1002E00000000000080075216C290D30A400A40B4B
:1002F0007729000008001030A8020001031C013E0D
:10030000A902031C080084290A30A8020001031C6A
:10031000013EA902031C080084292A088004200841
:10032000A8002108A9007B210130A202031CA3031D
:100330002A0980052008A8002108A9007B21A2081D
:0C034000031D8D29A308031D8D29080052
:02400E00C431BB
:00000001FF
